:020000040000FA
:0400000057EF00F0C6
:020008004FD0D7
:08001800D8CF01F1E8CF00F19F
:10002000E0CF02F104009DA802D09EB805D09DAAA1
:1000300002D09EBA14D031D013A304D001EE90F0B8
:10004000139302D02BC1E9FFEF6604D013979D985C
:100050009E9821D0EFCFADFFEE6A9E981CD09E9A5D
:10006000060EAB14D8A411D0606703D001EE60F087
:1000700002D02CC1E9FFAECFEEFF8F0EE96003D0B6
:100080000A0EAE6205D0138308D0AE50AB98AB8891
:10009000E9CF2CF102D0E9CF2BF102C1E0FF00C182
:1000A000E8FF01C1D8FF10001C2B9E921100010136
:1000B000F26A800ED06E720ED36E870ED56E320E3F
:1000C0009D6E010EA06E020E9F6EBF0E946EF19E8D
:1000D0000F0EC16EFF0E936E8068C2907F0E926EFF
:1000E000E10ED76E7B0ED66EF294F2A4FED7030E0D
:1000F000CA6E0C0EBA6E11EE00F0E66A400EE162B6
:10010000FCD711EE40F0156B152B15514FEC05F097
:10011000E66E100E156101D0F7D7240EAC6ECF0E2F
:10012000AF6E900EAB6E11EE60F0E66A900EE1627B
:10013000FCD73F0E086F06811399236B010E156FD4
:100140001551401503E0151D231702D01551231337
:10015000200E156102D01547F3D7D180460EBB6E35
:10016000BA98BA9A9E6AA16A9E9AF28EF28C04009C
:10017000E4EC00F001EC01F038EC01F076EC01F079
:10018000A9EC01F011EC02F0040081EC02F0C6ECE5
:1001900002F08CEC02F0EFEC02F000EC03F02DEC3E
:1001A00003F054EC03F0A3EC03F00400B5EC03F00F
:1001B000C8EC03F0E6EC03F053EC04F0BBEC04F005
:1001C00017EC05F0B7EF00F013B919D081BE17D0C6
:1001D00003B716D0FF0E206102D0202B11D081AEC4
:1001E00001D00DD0206B038703B106D003B308D034
:1001F00006A106D0038B04D00391038D01D0039791
:10020000120013B934D004B113D003AB30D04BC1BA
:1002100024F1039B04818050C00B806E11EE46F0E8
:10022000200E156F4B6106D015431551E12AFAD700
:10023000F2A41DD040C116F124511617161D8016C8
:100240002317241D7F0B9216010E24650AD0244328
:1002500064EC05F0E12A17C1D7FF18C1D6FFF2946C
:1002600006D0076B038104910A6B0B6B296B12009C
:1002700013B93BD004B309D003AD37D0010E246FBE
:10028000039D048311EE41F002D0F2A42ED024513C
:1002900092124B5124610AD0244764EC05F0E12A04
:1002A00017C1D7FF18C1D6FFF2941FD0405103A346
:1002B00005D03F0B236F05813F0E05D0401D3F0B3E
:1002C000236F0681000E076F0493CA9494822293D1
:1002D000229122952299229B22973F0E086F0A6B4A
:1002E0000B6B296B149B149D2A6B120081CF15F1A7
:1002F00003A505D015AD25D004A506D029D015BD80
:1003000020D004A501D024D0264B252B010E256535
:100310001FD0AA0E26651CD004854C6704D000D0DF
:1003200015AD09D002D015BD06D003B311D003839B
:10033000038F05910DD003A30BD00393038F069178
:1003400007D0256B266B15AD039515BD0385049568
:10035000120013B965D004B163D003A361D005B115
:100360005FD00A675DD00B675BD0296759D003AFB8
:100370000ED007C108F1039F0C6B059306930595FA
:10038000286B276B0B6B010E0F6F11EE41F00851BC
:100390000F1544E105B515D005B317D003A108D05A
:1003A00027510F150BE028510F1519E0286B276B0B
:1003B0000FC109F17BEC02F0058332D00FC127F1A8
:1003C0002FD0F2A42DD005952BD003A111D00F5121
:1003D0004D150EE00C510F150BE1F2A421D00F5179
:1003E0000A132289276727C129F1286B276B18D0A8
:1003F0000F5108134B510F610AD0059364EC05F0BF
:1004000017C1D7FF18C1D6FFF294058507D00E6B30
:100410000A6B0C6B05810593228102D00F47E12AFC
:10042000120013B967D003B365D006B163D00B6770
:1004300061D00A675FD003AF17D0071D3F0B086F6D
:10044000039F06910D6B069306950593286B276B0A
:100450004BC110F111EE46F0200E156F106104D063
:1004600015431551E12AFAD70851101541E106B597
:1004700015D006B317D003A108D0275110150BE0F3
:10048000285110151AE0286B276B10C109F17BEC7D
:1004900002F006832FD010C127F12CD0F2A42AD06D
:1004A000069528D003A10FD010514D150CE00D5129
:1004B000101509E1F2A41ED002D0286B276B105151
:1004C0000B13228917D010510813010E10650AD0A2
:1004D000069364EC05F017C1D7FF18C1D6FFF2945C
:1004E000068506D00E6B0B6B0D6B0681069302D052
:1004F0001043E12A1200F80ED76E5F0ED66EF2940A
:10050000120004B107D0095105E0801A071B231B14
:1005100009C10EF1096B120003A137D00B6735D06A
:100520000A6733D00E6701D030D00E514D152AE046
:100530000E51401514E105A309D00E518114D8B411
:1005400024D00E510C130E1D0A171CD00E5181140D
:10055000D8A41BD00E510D130E1D0B1713D005A3DD
:1005600009D00E518114D8A410D00E510C130E1DB9
:100570000A1708D00E518114D8B407D00E510D13AC
:100580000E1D0B170EC11FF10E6B120003A126D01A
:100590000B6724D00A6722D0276701D01FD02751CC
:1005A0004D1518E0275140150BE1275103A304D046
:1005B0008114D8A413D00ED08114D8B40FD00AD08F
:1005C000275103A304D08114D8B408D003D08114D8
:1005D000D8A404D027C128F1271D0B17120003A1AE
:1005E0000ED014BB03D014BD01D009D0F2A407D0A3
:1005F000212B2A2B670ED76E690ED66EF29412004D
:100600004EA32AD003A128D00A510B1125E122B113
:100610000AD022A321D003B30ED022B5CA9494826B
:100620002293229519D022832291216B670ED76ED7
:10063000690ED66E11D022B50FD04F29060DF3509A
:10064000216101D009D0330ECB6E1A0EBB6E9E9283
:10065000CC6ACA849492228512004EA524D022BB73
:1006600012D022B901D01FD01C6B1D6B330ECB6E84
:100670001A0EBB6E2299100E1E6F9E92CC6ACA840F
:100680009492228B10D00B510A1109E01E511C6369
:100690000AD0C80E1D6103D01D2B1C6B04D09E9286
:1006A000CA949482229B12004EA14CD003B102D076
:1006B0001F6B48D022BB46D022B703D01F670AD099
:1006C00041D01E511C633ED01F6B9E92CA949482EF
:1006D000229738D01C6B1D6B0F0EF76EE80EF66E6E
:1006E000F86A166B010E156F1F6504D0154715517A
:1006F000F62AFAD7800EA66E0800F5CF16F1162B53
:100700001643169F16C1BBFFF5CFCBFF080E166F21
:10071000010E156F1F51156103D01547162BFAD71F
:1007200003A304D04B51156306D003D0010E15630B
:1007300002D0163B228F16C11EF19E92CC6ACA844B
:1007400094922287120003A10FD00A510B110CE0E2
:1007500014AB04D0240E2A6104D006D02A6B148B6B
:1007600003D00391038D149B120003A110D003A3A7
:100770000DD005A10BD014AD04D0840E2A6104D095
:1007800006D02A6B148D03D00391038D149D1200A3
:10079000116B03B10CD004B10AD0070E1215070873
:1007A00006E0070E1215000802E0118104D003A331
:1007B000118303B3118511B1928E11B3809E11B7CD
:1007C000808E11B5807E11A1929E120013B96AD05D
:1007D00021EE5AF0010E156F5C6F5D6F5E6F5F6FFB
:1007E000DF6A03A106D00A510B11151502E0DF865E
:1007F00007D01551231502E0DF8202D0DF8400D03C
:100800004B51156103D01547D92AEAD7122B21EE97
:100810005AF0010E156F15BD28D0DFA003D0155179
:10082000941210D0151D9416DFA203D0151D821648
:1008300009D0DFA603D01551821204D0DFA402D064
:100840001551821A03B10CD004B30AD00F0E121541
:100850000F0806E00F0E1215000802E01551941261
:10086000D92A154715B31547D6D75FA102D0928C68
:100870000CD0929C5FA302D0809C07D05FA702D0CF
:10088000808C03D05FA50ED0807C03B10BD004B365
:1008900009D00F0E12150F0805E00F0E12150008F3
:1008A00001E0928C120013B765D013BB03D013B5CF
:1008B0003BD060D04D0E906F03C115F132EC05F0C6
:1008C00016C191F15AC115F132EC05F016C192F141
:1008D0005BC115F132EC05F016C193F15CC115F165
:1008E00032EC05F016C194F15DC115F132EC05F062
:1008F00016C195F15EC115F132EC05F016C196F105
:100900005FC115F132EC05F016C197F122C115F166
:1009100032EC05F015C198F10D0E996F0A0E9A6F21
:10092000000E9B6F229F21D0176B11EE40F021EE3D
:1009300090F0500EDE6E020E156F32EC05F015C110
:10094000DEFF16C1DEFF172BE6CF15F132EC05F006
:1009500015C1DEFF16C1DEFF100E1763F4D70D0EB2
:10096000DE6E0A0EDE6E000EDE6E13831395139B91
:1009700013879D88120013B758D013A356D09D9AA1
:100980004D0E606306D0138B1393606B616B626BCB
:100990004CD0550E605D06E0530E605D03E0520ED4
:1009A000605D3CE104B342D003A103D00391038D09
:1009B0003DD0176B138911EE40F021EE60F0DECFD1
:1009C00016F1550E166321D0000E2D6BDE502D272B
:1009D000810ED962FBD7DECF15F1DECF16F141ECE7
:1009E00005F015512D631AD021EE61F0176B172B0E
:1009F000DECF15F1DECF16F141EC05F015C1E6FFB3
:100A0000100E1763F4D7148109D0530E166302D069
:100A1000138504D0520E166301D0FF00139321EE0C
:100A200060F0DE6A800ED962FCD79D8A120014A1A4
:100A300018D013B716D011EE40F0000E1B6302D091
:100A4000166B03D01B51E6CF16F155EC05F00400F0
:100A5000A6B2FDD7100E1B6102D01B2BEED714914E
:100A60001B6B12003A0E1A6F15510F0B300F1A65DF
:100A7000070F166F15390F0B300F1A65070F156F1B
:100A800012000A0E1A6F300E155D1A65F90F156FF8
:100A9000153B300E165D1A65F90F15271200A96E69
:100AA000A69CA69EA680A8501200A96E16C1A8FFFB
:100AB000A69CA69EA684F29E550EA76EAA0EA76EB1
:100AC000A682A694F28E12000F0EF76EC00EF66E7E
:100AD000F86AE744FE0BF626800EA66E0900F5CFF5
:0A0AE00018F10800F5CF17F112001D
:100FC00064FF16FFC8FE79FE2BFEDDFD8FFD41FD9F
:100FD000F3FC6CFBE5F95FF8D8F6CBF3BEF0B0EDAF
:0E0FE000A3EA96E789E47BE1EED4BDB29E8DD4
:020000040030CA
:0E000000FF38F7E0FFFDFAFFFFFFFFFFFFFFF5
:0200000400F00A
:10000000000008080808080808080808200100037C
:1000100007FFFFFFFFFFFFFFFFFFFFFFFFFFFFFFE8
:10002000FFFFFFFFFFFFFFFFFFFFFFFFFFFFFFFFE0
:10003000FFFFFFFFFFFFFFFFFFFFFFFFFFFFFFFFD0
:10004000FFFFFFFFFFFFFFFFFFFFFFFFFFFFFFFFC0
:10005000FFFFFFFFFFFFFFFFFFFFFFFFFFFFFFFFB0
:10006000FFFFFFFFFFFFFFFFFFFFFFFFFFFFFFFFA0
:10007000FFFFFFFFFFFFFFFFFFFFFFFFFFFFFFFF90
:10008000FFFFFFFFFFFFFFFFFFFFFFFFFFFFFFFF80
:10009000FFFFFFFFFFFFFFFFFFFFFFFFFFFFFFFF70
:1000A000FFFFFFFFFFFFFFFFFFFFFFFFFFFFFFFF60
:1000B000FFFFFFFFFFFFFFFFFFFFFFFFFFFFFFFF50
:1000C000FFFFFFFFFFFFFFFFFFFFFFFFFFFFFFFF40
:1000D000FFFFFFFFFFFFFFFFFFFFFFFFFFFFFFFF30
:1000E000FFFFFFFFFFFFFFFFFFFFFFFFFFFFFFFF20
:1000F000FFFFFFFFFFFFFFFFFFFFFFFFFFFFFF020D
:00000001FF
